:020000040800F2
:10000000E829002085010008851D00086D180008FA
:10001000811D0008B7020008DD5400080000000040
:10002000000000000000000000000000C5200008E3
:100030004B0F0008000000008D1E00084927000833
:100040009F0100089F0100089F0100089F01000810
:100050009F0100089F0100089F0100089F01000800
:100060009F0100089F0100089F0100089F010008F0
:100070009F0100089F0100089F0100089F010008E0
:100080009F0100089F0100089F0100089F010008D0
:10009000BD0200089F010008D90200089F01000866
:1000A0009F0100089F0100089F0100089F010008B0
:1000B0009F0100086D2800089F0100089F010008AB
:1000C0009F0100089F0100089F0100089F01000890
:1000D0009F0100089F0100089F0100089F01000880
:1000E0009F0100089F0100089F0100080000000018
:1000F0000000000000000000000000000000000000
:1001000000000000000000009F0100089F0100089F
:100110009F0100089F0100089F0100089F0100083F
:100120009F0100089F0100089F0100089F0100082F
:100130009F0100089F0100089F0100089F0100081F
:100140009F01000879040008AD0400089F01000821
:10015000DFF80CD000F068F800480047ED570008C1
:10016000E8290020EFF30980704780F30988704781
:10017000EFF30880704780F30888704740BA7047F3
:10018000C0BA70470648804706480047FEE7FEE7CA
:10019000FEE7FEE7FEE7FEE7FEE7FEE7FEE7FEE737
:1001A000012800085101000810B5431A934209D2F2
:1001B0008318881803E010F8011D03F8011D521E72
:1001C000F9D210BD40EA01039B0703D009E008C93A
:1001D000121F08C0042AFAD203E011F8013B00F80C
:1001E000013B521EF9D210BDD2B201E000F8012B42
:1001F000491EFBD270470022F6E710B513460A46A7
:1002000004461946FFF7F0FF204610BD30B50446FE
:100210000020034600E05B1C934203D2E05CCD5C0F
:10022000401BF8D030BD0000064C074D06E0E068EA
:1002300040F0010394E8070098471034AC42F6D32D
:10024000FFF78AFF085C0008285C000870B58C186E
:1002500010F8015B15F0070301D110F8013B2A11DA
:1002600006D110F8012B03E010F8016B01F8016BC7
:100270005B1EF9D12B0705D40023521E0DD401F8C3
:10028000013BFAE710F8013BCB1A921C03E013F88C
:10029000015B01F8015B521EF9D5A142D8D30020C1
:1002A00070BD10B501214FF0C05001F015FE0120C6
:1002B00001F0BCFD10BD00BFFEE7000000B585B039
:1002C000002005F0D7F96A460021024800F095FBAE
:1002D00005B000BD0064004010B54FF40071154832
:1002E00000F068FA01280DD11349124800F026FAEF
:1002F000012802D1002005F079F94FF400710D4872
:1003000000F028F94FF480610A4800F053FA012800
:100310000ED10949891C074800F010FA012802D1C2
:10032000002005F077F94FF48061024800F012F9DF
:1003300010BD0000006400400200F01000B589B05C
:100340000121092001F0E8FD0121480601F0C4FD6A
:100350000121880601F0C0FD4FF40050ADF82000E7
:1003600003208DF8220018208DF8230008A94048AA
:1003700000F029FF4FF48050ADF8200048208DF8A0
:10038000230008A93A4800F01EFF00208DF81A004B
:1003900001208DF81B0000208DF81C008DF81D0039
:1003A0008DF81E008DF81F008DF8160001208DF8C5
:1003B000170008208DF8180001208DF8190006207C
:1003C000ADF8140005A92B4800F08DFA0E208DF829
:1003D0000E0000208DF80F0001208DF81000002085
:1003E000ADF80400ADF80600ADF80800ADF80A005D
:1003F0000120ADF80C008DF8110001A800F01AF9E9
:10040000012210211B4800F065FA41208DF8000000
:1004100001208DF8010000208DF8020001208DF8E8
:100420000300684601F0B6FC012005F017F901222F
:100430005102104800F04EFA012291020D4800F0DE
:1004400049FA0122D1030B4800F044FA42208DF80A
:10045000000001208DF8010000208DF8020001202D
:100460008DF80300684601F095FC002009B000BD3E
:10047000000C01400068004010B586B00024012047
:1004800005F0F8F801AA0121074800F0B6FA05982E
:10049000009001A80FC804F0DDFE142101A8FFF7A9
:1004A000AAFE06B010BD00000068004010B54FF471
:1004B0000071184800F07EF9012810D1164915483E
:1004C00000F03CF9012805D105F090F812491148D7
:1004D00000F024F84FF400710E4800F03BF84FF4A0
:1004E00080610C4800F066F9012812D10A49891C84
:1004F000084800F023F9012806D105F08BF80649D9
:10050000891C044800F00AF84FF48061014800F0AB
:1005100021F810BD006800400200F01000220C4BD2
:10052000994202D10023836111E0C1F3130201F06B
:1005300000730BB1C2600AE001F080630BB102618D
:1005400005E001F000630BB1826000E0426070479B
:100550007000F030B1F5007F3AD00FDC202928D0B0
:1005600006DC01291CD004291DD0082940D11DE03A
:10057000402921D0B1F5807F3AD126E0B1F5004F76
:1005800031D006DCB1F5806F25D0B1F5006F2FD1E9
:1005900024E0B1F5803F12D0B1F5003F28D111E041
:1005A000154A826025E00822C26022E01022C26063
:1005B0001FE0082202611CE01022026119E00822FB
:1005C000426016E01022426013E00422426010E014
:1005D000042242600DE0042242600AE000228261AF
:1005E0000422426005E0002282610422426000E0B1
:1005F00000BF00BF704700000101010010B50446B4
:100600000B48844209D10121480601F075FC002104
:100610004FF0007001F070FC08E00121880601F045
:100620006BFC00214FF0806001F066FC10BD000003
:100630000064004010B50021837A012202FA03F120
:100640003D4A126842F001023B4B1A603A4A1C32A2
:1006500012688A43384B1C331A60027BCAB9364A87
:100660000C3212688A43344B0C331A604288C388B8
:1006700042EA0343304A4032847A42F834300288F6
:10068000838842EA03432C4A4032847A02EBC40254
:100690005360027B012A19D1274A0C3212680A439F
:1006A000254B0C331A604288038842EA0343224AEE
:1006B0004032847A42F83430C288838842EA034365
:1006C0001D4A4032847A02EBC4025360C27A3AB9BE
:1006D000194A121D12688A43174B1B1D1A6006E047
:1006E000154A121D12680A43134B1B1D1A6002891A
:1006F00032B9114A143212688A430F4B14331A600C
:100700000289012A06D10C4A143212680A430A4BA4
:1007100014331A60427B012A06D1074A1C32126840
:100720000A43054B1C331A60034A126822F0010287
:10073000014B1A6010BD00000066004010B5024673
:10074000002001F4700343B19369C1F31304234003
:100750000BB101202DE000202BE001F0807343B1AC
:100760005368C1F3130423400BB1012021E00020A2
:100770001FE001F0006343B19368C1F31304234009
:100780000BB1012015E0002013E001F0007343B12C
:10079000D368C1F3130423400BB1012009E000200A
:1007A00007E01369C1F3130423400BB1012000E0FB
:1007B000002010BD70B504460D4600266069284033
:1007C000002871D0B5F5807F5CD010DC082D35D0C5
:1007D00006DC012D20D0022D24D0042D72D127E07B
:1007E000102D31D0202D35D0402D6BD138E0B5F50E
:1007F000004F60D009DCB5F5007F49D0B5F5806FBA
:100800004CD0B5F5006F5DD14FE0B5F5803F2DD0F0
:10081000B5F5003F56D12FE0A0682D4900F0ECFA65
:10082000064651E0E068032100F0E6FA06464BE098
:10083000E068082100F0E0FA064645E0E068102193
:1008400000F0DAFA06463FE02069032100F0D4FA0E
:10085000064639E02069082100F0CEFA064633E06A
:100860002069102100F0C8FA06462DE060680821D2
:1008700000F0C2FA064627E06068102100F0BCFADA
:10088000064621E0A069012100F0B6FA06461BE009
:10089000A069022100F0B0FA064615E0A069042123
:1008A00000F0AAFA06460FE00FE0A069702100F000
:1008B000A3FA064608E06068042100F09DFA0646A7
:1008C00002E0FFE7002600BF00E00026304670BDD2
:1008D000010101001AB143690B43436102E043691E
:1008E0008B434361704730B50246002000231468F3
:1008F00024F002041460146844F00104146000E061
:100900005B1C546804F001041CB94FF6FF74A34249
:10091000F6D1546804F001040CB900206CE08C7925
:10092000012C04D1146844F08004146003E01468BE
:1009300024F080041460CC79012C04D1146844F0B4
:100940004004146003E0146824F0400414600C7A3E
:10095000012C04D1146844F02004146003E01468EE
:1009600024F0200414604C7A012C04D1146844F063
:100970001004146003E0146824F0100414608C7AEE
:10098000012C04D1146844F00804146003E01468D6
:1009900024F008041460CC7A012C04D1146844F0CB
:1009A0000404146003E0146824F0040414608C78D8
:1009B000A407CD7844EA05640D7944EA05444D79ED
:1009C00044EA05540D886D1E2C43D461146824F04C
:1009D00001041460002300E05B1C546804F001046F
:1009E0001CB14FF6FF74A342F6D1546804F0010421
:1009F0000CB1002000E0012030BD10B500F5D87327
:100A000003EB01131B6803F004031372137A53B949
:100A100000F5D87303EB01131B6840F2FF7404EA7E
:100A20005353136009E000F5D87303EB01131B68FF
:100A30006FF0604404EAD303536000F5D87303EB0E
:100A400001131B6803F00203537200F5D87303EB24
:100A500001135B6803F00F03937200F5D87303EB87
:100A600001135B681B0AD37400F5D87303EB011301
:100A70009B68D37200F5D87303EB01139B681C0AC3
:100A8000147300F5D87303EB01139B681C0C5473AB
:100A900000F5D87303EB01139B681B0E937300F5ED
:100AA000D87303EB0113DB68D37300F5D87303EB42
:100AB0000113DB681C0A147400F5D87303EB0113EF
:100AC000DB681C0C547400F5D87303EB0113DB686E
:100AD0001B0E937421B9C36843F02003C36003E085
:100AE000036943F02003036110BD10B502460020E6
:100AF000936803F08063B3F1806F00D110E09368D6
:100B000003F00063B3F1006F01D1012008E09368A6
:100B100003F08053B3F1805F01D1022000E0042094
:100B2000042874D002F5C07303EB00131B6803F0B4
:100B3000010402F5C07303EB00131C600B7A7BB950
:100B40004B7A0C8843EA445302F5C07404EB00145A
:100B50002468234302F5C07404EB0014236010E002
:100B60000B7A4C6843EAC4034C7A234302F5C07401
:100B700004EB00142468234302F5C07404EB001452
:100B800023608B7A03F00F038B7202F5C07303EBC3
:100B900000135B6823F00F0402F5C07303EB00132E
:100BA0005C6002F5C07303EB00135B688C7A23432F
:100BB00002F5C07404EB001463608B7B1C064B7B56
:100BC00044EA03440B7B44EA0323CC7A234302F533
:100BD000C07404EB0014A3608B7C1C064B7C44EABD
:100BE00003440B7C44EA0323CC7B234302F5C0740B
:100BF00004EB0014E36002F5C07303EB00131B6801
:100C000043F0010402F5C07303EB00131C6010BD38
:100C100010B50246002321B1012907D002290FD1C6
:100C200009E090681D4C00EA04030BE090681C4C3E
:100C300000EA040306E090681A4C00EA040301E0AD
:100C4000002300BF00BF184C181BA34216D007DCBE
:100C500083B16FF08060184470B1022818D111E0A0
:100C6000B0F5007F10D0114C204448B1B0F5003FE2
:100C70000ED10BE002230DE000230BE0002309E07E
:100C8000002307E0012305E0012303E0012301E045
:100C9000002300BF00BFD8B210BD00000300000455
:100CA0000003000800000310000100080001FFF726
:100CB0004FF6FF710180704770B50B4600210BE0C5
:100CC0005D5C068885EA2624054D35F814500678C3
:100CD00085EA06250580491C9142F1D370BD0000CC
:100CE00056590008F0B504460D462946204600F046
:100CF00009F80746615D681C205C41EA002686EA27
:100D00000700F0BD70B502464FF6FF7048F20505CA
:100D100017E0491E12F8014B80EA042000230EE080
:100D200000F400462EB14FF6FF7606EA4000684018
:100D300003E04FF6FF7606EA40005E1CF3B2082B94
:100D4000EEDB0029E5D170BD30B50B46002104E093
:100D50005D5C04682C440460491C9142F8D330BDAA
:100D60000FB430B585B00024142208A96846FFF7F7
:100D70001BFA012004F092FC20B9012005B030BC20
:100D80005DF814FB69460E48FFF7AFFE05460024E8
:100D900001E0601C84B2012004F080FC40B12946CF
:100DA0000748FFF735FF18B940F6FF708442F0DBC3
:100DB00040F6FF70844201DB0120DFE70020DDE721
:100DC00000680040002001207047000010B509486D
:100DD000407801280CD107488078012808D10020EC
:100DE00004494870887000F03DFD012001494871B8
:100DF00010BD0000141F00200246002002EA01037B
:100E00000BB1012000E000207047000000200349E2
:100E10000978C1F3800101B101207047D706002095
:100E2000002003490978C1F3400101B10120704756
:100E3000D706002010B5034600202AB18B4201D00E
:100E4000012006E0002004E08B4201D1012000E0F7
:100E5000002010BD01460020064A128A8A4207D0AF
:100E6000044A528A8A4203D0024A12888A4200D136
:100E7000012070478A5B000801460020012901D04B
:100E8000032900D1012070470146002001F08002B3
:100E900002B901207047024600208A4200D1012099
:100EA000704700000020054A937B527B03EB02222F
:100EB00091B2502900DC012070470000D7060020C5
:100EC000002002490880091D08807047B06C00406E
:100ED0002DE9F8436946164800F088F8DFF8549089
:100EE000002420E0144931F8140000F0CFFA054640
:100EF000FF2D16D0114830F8150000EB09081048F6
:100F000030F814600F4830F8140000994718314643
:100F10003846FFF7E7FE20B9324639464046FFF72C
:100F200043F9601CC4B20A2CDCDBBDE8F883000086
:100F3000681F002030060020E65B0008565B0008B2
:100F4000D25B0008BE5B00087047704710B50446CE
:100F500006E0142004F0C4FA00F080FD601E84B2A4
:100F6000002CF6DC10BD00002DE9F84F83464FF051
:100F7000000A00200090584600F09CFA8046B8F124
:100F8000FF0F27D0584600F081FA0546FF2D21D0EB
:100F90001148445DDFF84490114830F8150000EB2B
:100FA000090621463046FFF7ADFE87B23755641C6F
:100FB00038123055641C0B4830F818000A4900EB11
:100FC000010ABAF1000F05D00023224631465046EF
:100FD00000F01EF8BDE8F88F785B000830060020AE
:100FE000565B0008BE5B0008681F002002460748E9
:100FF000904201D1086007E004484038904201D196
:10100000086001E0002070470120FCE7A81F0020D5
:101010002DE9F04104460D4616461F463B46324632
:101020002946204604F076FC0120BDE8F0812DE938
:10103000F04104460E4600270025C4F30A0010B113
:101040000120BDE8F08100F09FF8352000F014F891
:10105000254608E0284600F015F8042801D00127AD
:1010600004E005F50065A019A842F3D800BF00F020
:1010700049F83846E5E700000149C86070470000BC
:101080000020024030B5044604250F4800F088F8DF
:101090000546042D16D10D48006940F002000B49A9
:1010A000086108464461006940F040000861064854
:1010B00000F076F805460548006941F6FD710840E4
:1010C00002490861284630BDFFFF0F0000200240A2
:1010D00004200B49C96801F0010109B101200EE0AB
:1010E0000749C96801F0040109B1022007E0044979
:1010F000C96801F0100109B1032000E00420704725
:10110000002002400348006940F080000149086166
:10111000704700000020024078B506460C460425C2
:10112000002000904FF6FF7000F03AF80546042DBD
:1011300026D11448006940F001001249086134804A
:101140004FF6FF7000F02CF80546042D11D1B01CAD
:101150000090200C009908804FF6FF7000F020F8F6
:1011600005460848006941F6FE71084005490861D6
:1011700006E00448006941F6FE7108400149086133
:10118000284678BD002002400248034948600348D1
:10119000486070472301674500200240AB89EFCDCE
:1011A00000B502460423FFF793FF034603E0FFF771
:1011B0008FFF0346521E012B01D1002AF7D102B93D
:1011C0000523184600BD2DE9F04102460025002602
:1011D000002000230024002791F803C00CF00F0525
:1011E00091F803C00CF0100CBCF1000F03D091F883
:1011F00002C04CEA050591F800C0BCF1000F31D0E7
:10120000146800202BE04FF0010C0CFA00F3B1F849
:1012100000C00CEA03069E4220D183004FF00F0C61
:101220000CFA03F7BC4305FA03FC4CEA040491F8FA
:1012300003C0BCF1280F06D14FF0010C0CFA00FCE2
:10124000C2F814C00AE091F803C0BCF1480F05D100
:101250004FF0010C0CFA00FCC2F810C0401C08282A
:10126000D1D31460B1F800C0BCF1FF0F34DD546875
:1012700000202EE000F1080C4FF0010808FA0CF3F2
:10128000B1F800C00CEA03069E4221D183004FF062
:101290000F0C0CFA03F7BC4305FA03FC4CEA0404F8
:1012A00091F803C0BCF1280F05D100F1080C08FA31
:1012B0000CF8C2F8148091F803C0BCF1480F07D1B4
:1012C00000F1080C4FF0010808FA0CF8C2F8108081
:1012D000401C0828CED35460BDE8F081F0B50A4622
:1012E000002300240021002500F00046B6F1004F45
:1012F00002D11D4EF16901E01B4E7168C0F3034538
:1013000083B200F44016B6F5401F08D121F0706199
:10131000154E766826F07066134F7E6012E000F47A
:101320008016B6F5801F06D1032606FA05F4A14300
:1013300041F0706106E0460D360103FA06F6B1434E
:1013400041F0706122B1460D360103FA06F63143D1
:1013500000F00046B6F1004F02D1034EF16101E00A
:10136000014E7160F0BD0000000001404161704716
:101370000161704718B501460C128DF80040CCB2DF
:101380008DF801404FF6FE70002221E01DF802406A
:1013900080EA0420002317E000F4004474B100F058
:1013A00080042CB148F2084484EA4004A0B209E069
:1013B00048F2250484EA4004A0B203E04FF6FF742B
:1013C00004EA40005C1CE3B2082BE5DB541CE2B2EB
:1013D000022ADBDB18BD70B5044603F013FF45435A
:1013E0002570280C6070002070BD00002DE9F047CA
:1013F000064600240027204890F82A001E4991F84C
:10140000291000EB012087B262222146641C72542D
:101410003A0A2146641C72542146641C7754DFF852
:101420005C90002507E0164830F81500B84200D15E
:1014300003E0681CC5B2112DF5DB00BF112D01D1F1
:10144000022404E03846FFF705FD00B90224022C0F
:101450000ED00C4810F805800B4A32F8152002EB2C
:10146000090130194246FEF79FFE04EB080084B2E2
:101470002046BDE8F0870000141F00203006002041
:101480008A5B0008785B0008565B00080246FF2074
:10149000002108E0064B33F81130934201D1084691
:1014A00003E04B1CD9B21129F4D300BF70470000F0
:1014B0008A5B00080246FF20002108E0064B33F853
:1014C0001130934201D1084603E04B1CD9B20A29DE
:1014D000F4D300BF70470000E65B000804480078C2
:1014E00020B1002002490870012070470020FCE76D
:1014F0005800002006480068064908600448001F9C
:10150000006848600248083800688860704700003A
:10151000F0F7FF1F600100205C480088401C80B28B
:101520005A4908800A2872DB002008805848C08F7A
:10153000B0F5FA7F2FDA5648C08F401C5449C8874F
:101540000846C08FB0F5FA7F25D100200872084602
:10155000C07E032803D00846C07E02281BD100208D
:101560004B4988760120C876002081F820008871D8
:10157000C88781F8220081F8230081F82500C8730C
:1015800044480079012803D100204249C8820871EB
:1015900001203F49087040480088401C80B23E4905
:1015A0000880642800DA704700203B4908803848EA
:1015B00090F82700D8B1364890F82700401E3449EB
:1015C00081F82700084690F8270080B90846C078BF
:1015D00001280CD10020C870084690F82600002889
:1015E00005DD084690F82600401E81F826002848B0
:1015F00090F8220060B12948007820F001002749C6
:1016000008700846007820F0020008700DE03AE00B
:101610002248007820F00100401C2049087008464C
:10162000007820F00200801C0870194890F8230010
:1016300058B11A48007820F004001849087008468C
:10164000007820F0080008700CE01448007820F0C2
:101650000400001D114908700846007820F00800B9
:10166000083008700A48007A30B10C48007820F041
:1016700010000A49087006E00848007820F01000C1
:1016800010300649087000BF8DE700002E010020D1
:10169000141F0020E01600202C0100206C00002008
:1016A0007047704770B505460E460848067000241E
:1016B00004E0285D06490855601CC4B20348007860
:1016C0008442F6DB01F092F970BD00003901002080
:1016D000300100200146002004E0054A125C0A5453
:1016E000421CD0B2034A12789042F6DB70470000E9
:1016F000300100203901002070B504460D4601F08C
:1017000081FA064632462946204603F0C7FC70BDE2
:1017100070B505460E4608480670002404E0285DB2
:1017200006490855601CC4B2034800788442F6DBC1
:1017300001F0E0F970BD0000390100203001002007
:1017400010B501F0F1FA10BD10B5044603F03AFDF2
:1017500000200149087010BD3801002001480078C0
:1017600070470000390100207FB505460E4800682B
:1017700000900E4800788DF80400002405E0295DF3
:101780000DF105000155601CC4B208480078844280
:10179000F5DB01208DF80D00054948709DE80F002C
:1017A00002F08AFB7FBD00003C0100203A010020CE
:1017B000141F002001490870704700003A01002002
:1017C00020B940F27F71044A116003E040F27F715A
:1017D000014A1160704700003C0100207047000082
:1017E0002DE9F04105460E4601F00CFA04460A4880
:1017F000007878B97F2020706570A67003270020DC
:10180000FFF7DEFF01F0F4FD384601F05BFA01203E
:1018100001490870BDE8F081380100202DE9F04150
:1018200005460E4601F0EEF980460D480078A8B94D
:10183000A5B1002404E0305D08F80400601C84B207
:10184000AC42F8DB2F460020FFF7BAFF01F0D0FDD5
:10185000384601F037FA012001490870BDE8F081EF
:101860003801002010B501F063F810BD00BFFEE79D
:1018700010B54FF400600B49086003F0B0FF4FF45F
:1018800080600849091F086003F0A9FF4FF48060D9
:101890000449086003F0A3FF4FF400600149091FE9
:1018A000086010BD140C014010B54FF400600949E8
:1018B000086003F094FF4FF480600649086003F06D
:1018C0008EFF4FF480600349091D086003F087FF15
:1018D00010BD0000100C014070B505460024002624
:1018E00018E06006040E4FF480600F49086003F0B2
:1018F00076FF0D480838006800F4006008B1601CED
:10190000C4B24FF480600849091D086003F067FF06
:10191000701CC6B2082EE4DB15B9FFF7C5FF01E065
:10192000FFF7A6FF204670BD100C014070B50446BD
:10193000002524E004F0800020B14FF4006011493C
:10194000086004E04FF400600E49091D086003F0D0
:1019500046FF4FF480600B49086003F040FF4FF4EE
:1019600080600849091D0860072D02D14000091F49
:1019700008606006040E03F032FF681CC5B2082D33
:10198000D8DB70BD100C014010B54FF400600A495F
:1019900008604010086003F022FF4FF40060064921
:1019A000091D086003F01BFF4FF480600249091D08
:1019B000086003F014FF10BD100C014010B54FF487
:1019C0000060074908604010091F086003F007FF26
:1019D0004FF400600249091F086003F000FF10BDCA
:1019E000140C014010B54FF400600E49086003F07C
:1019F000F6FE4FF480600B49086003F0F0FE0948E2
:101A00000838006800F4006008B1012400E00024F8
:101A10004FF480600349091D086003F0E0FE204692
:101A200010BD0000100C014070B505460C4645F293
:101A3000555000F033F8284600F024F8204600F016
:101A400027F800F017F800F001F870BD4CF6CC4014
:101A500001490860704700000030004010B500F0F8
:101A600009F810BD10B540F635410420FFF7DCFF42
:101A700010BD00004AF6AA20014908607047000026
:101A800000300040014948607047000000300040CD
:101A9000014988607047000000300040014908603B
:101AA00070470000003000402DE9F0472D480468E1
:101AB0002D48844201D0BDE8F0872A48001D046803
:101AC000B4F5205F02D3B4F5D03F00D9F3E7A60800
:101AD00004F0030000B1761CDFF89080244DFFF77E
:101AE00053FB002724E04FF0000AD8F80040C5F36C
:101AF0000A0010B92846FFF7C5FA0EE0214628462D
:101B0000FFF70AFB042800D108E00AF1010000F009
:101B1000FF0ABAF1030F00DB00E0EFE700BFD5F8E2
:101B200000904C4500D005E008F104082D1D7F1CF5
:101B3000B742D8D300BF0B48FFF7A4FAFFF7E2FA89
:101B40000B4840680B490860084600680A4908606D
:101B500007490868FEF70FFB07480068804700BF89
:101B6000A9E700000058020844332211006002086F
:101B70000080000818000020140000200020054A02
:101B80001188121F128842EA0141034A914200D192
:101B900001207047B46C00405CBA55AA10B572B60B
:101BA000FFF782FFFFF7EAFF28B101200F49087015
:101BB000FFF786F917E00E4800680E490840B0F1BB
:101BC000005F10D100F022FD094840680A49086012
:101BD000084600680949086005490868FEF7CBFA1D
:101BE00006480068804762B610BD0000580000201B
:101BF000008000080000FE2F600000205C00002034
:101C000008B501211C2000F087F94FF40070ADF8F1
:101C1000000010208DF8030003208DF802006946B3
:101C20005348FFF7D0FA4FF400715148FFF7A0FB7B
:101C30000120ADF8000010208DF8030003208DF87E
:101C4000020069464A48FFF7BEFA01214848FFF7FB
:101C50008FFB40F20240ADF8000010208DF8030029
:101C600003208DF8020069464148FFF7ACFA0221D3
:101C70003F48FFF77DFB4FF480613D48FFF776FB5F
:101C8000A020ADF8000010208DF8030003208DF88F
:101C9000020069463748FFF796FA20213548FFF7DA
:101CA00065FB80213348FFF763FB44F22720ADF842
:101CB000000010208DF8030003208DF80200694613
:101CC0002D48FFF780FA4FF400712B48FFF750FBC7
:101CD00001212948FFF74AFB02212748FFF746FB6D
:101CE00004212548FFF742FB4FF480412248FFF7CB
:101CF0003DFB20212048FFF739FB4FF48070ADF801
:101D0000000048208DF8030069461948FFF75BFA88
:101D10004FF40070ADF8000048208DF803006946CC
:101D20001448FFF750FA0121084600F0F5F80121A8
:101D30001248FFF7D3FA1020ADF8000001208DF80B
:101D4000020010208DF8030069460B48FFF73BFAAC
:101D500010210948FFF70CFB4FF40050ADF80000CC
:101D600004208DF8030069460248FFF72CFA08BDED
:101D70000008014000100140000C0140000130004B
:101D800000BFFEE7704710B54FF4A06000F03AF8CE
:101D900010BD000070B5002100230F22C47804B3E9
:101DA000154C246804F4E064C4F5E064210AC1F130
:101DB0000403CA40447804FA03F1847814402143B0
:101DC00009010E4C0678A155047804F01F05012482
:101DD000AC4005786D11AD0005F1E025C5F8004176
:101DE00009E0047804F01F050124AC40044D067896
:101DF000761145F8264070BD0CED00E000E400E0EF
:101E000080E100E002490143024A1160704700008E
:101E10000000FA050CED00E010B54FF4007200214F
:101E2000014803F0DAF910BD681F0020014908627B
:101E30007047000000000E421FB5012012490872D1
:101E40000020C8870098A0F2777010B1682818D1D8
:101E50000BE040F277700C49A1F84C009DF804109B
:101E60000DF10500FFF754FC0CE040F2DF7006496D
:101E7000A1F84C009DF804100DF10500FFF712FCCD
:101E800000E000BF00BF1FBD141F002070472DE9F8
:101E9000F04106460C4617464FF000080025FFF7B4
:101EA00073F93520FFF7E8F835460CE0284621683D
:101EB000FFF732F928682168884202D04FF0010804
:101EC00004E02D1D241DF019A842EFD800BFFFF734
:101ED00019F94046BDE8F08129B1064AD2690243AA
:101EE000044BDA6104E0034AD2698243014BDA61B0
:101EF000704700000010024029B1064A12690243EF
:101F0000044B1A6104E0034A12698243014B1A61CF
:101F1000704700000010024029B1064A926902434E
:101F2000044B9A6104E0034A92698243014B9A612F
:101F300070470000001002402DE9F041002100220E
:101F4000002500230026002400278C46DFF860814E
:101F5000D8F8048008F00C0121B1042907D0082921
:101F600059D109E0DFF84C81C0F8008058E0DFF873
:101F70004481C0F8008053E0DFF83481D8F8048051
:101F800008F47012DFF82881D8F8048008F480354E
:101F9000920C0D2A01D0921C00E0062235B9DFF820
:101FA000188102FB08F8C0F8008033E0DFF80081F8
:101FB000D8F82C8008F48036DFF8F480D8F82C802C
:101FC00008F00F0808F1010446B9DFF8E880B8FB13
:101FD000F4F808FB02F8C0F800801BE0DFF8D080BE
:101FE000D8F82C80C8F3031808F10107DFF8C08087
:101FF000D8F82C80C8F3032808F1020CDFF8B4806D
:10200000B8FBF7F808FB0CF8B8FBF4F808FB02F88B
:10201000C0F8008004E0DFF89C80C0F8008000BFBA
:1020200000BFDFF88C80D8F8048008F0F0010909BF
:10203000DFF8888018F80130D0F8008028FA03F81B
:10204000C0F80480DFF86880D8F8048008F4E06104
:10205000090ADFF8688018F80130D0F8048028FAFF
:1020600003F8C0F80880DFF84880D8F8048008F446
:102070006051C90ADFF8448018F80130D0F80480B4
:1020800028FA03F8C0F80C80DFF82480D8F8048020
:1020900008F44041890BDFF8288018F80130D0F8A7
:1020A0000C80B8FBF3F8C0F81080BDE8F0810000A8
:1020B0000010024000127A0000093D004300002099
:1020C00053000020704700002DE9F04104460D4602
:1020D000002700266078217800EB012086B21A489C
:1020E000008AB04211D11948007AA8420BD1184891
:1020F00090F8200028B12A46A11C1648FEF754F893
:102100001BE0332719E0132717E00F48408AB0423D
:1021100012D10E48407AA8420CD10D4890F8200008
:1021200030B12A46A11C0B480E30FEF73DF804E002
:10213000332702E0132700E0312717B93046FEF7B6
:1021400013FF3846BDE8F0818A5B0008785B000821
:10215000141F0020AA0600202DE9F04F8DB0044680
:1021600091469A464FF0000BD846002500260027DE
:10217000F048B0F84000042803DA13200DB0BDE8A1
:10218000F08F94F80080A078617840EA01257122F0
:102190003046711C8EB20DF8002022783046711C3A
:1021A0008EB20DF8002062783046711C8EB20DF8A8
:1021B0000020A2783046711C8EB20DF80020B8F1D4
:1021C000010F71D1DB49B1F840000621FEF763FE33
:1021D00018B14DF60420854215D0D649B1F840001B
:1021E0000C21FEF758FE10B1B5F57F4F0BD0D14949
:1021F000B1F840000E21FEF74EFE00287AD04FF6CF
:10220000017085427ED1CB4890F82000002876D01E
:10221000A5F55A40043830B1A0F51050FC38B8B1DB
:1022200001286AD141E0C44890F8300803280CD155
:102230002079E17800EB0120BF49888201273046F0
:10224000711C8EB20DF8007001E04FF0220B55E0CA
:10225000E0780006217900EB0140617900EB012074
:10226000A1790844B449C860E0790006217A00EBFE
:102270000140617A00EB0120A17A0844AE4908616F
:102280000846C068AD49884206D04FF0720B012065
:10229000A94981F8280806E04FF0780B0120A649EB
:1022A000087081F8240829E03DE0E07800062179F3
:1022B00000EB0140617900EB0120A1790844A049BD
:1022C0000860E0790006217A00EB0140617A00EBBA
:1022D0000120A17A08449B490860207BE17A00EB49
:1022E00001209949088001273046711C8EB20DF8F3
:1022F000007003E006E002E0FFE700BF0EE14FF0F0
:10230000330B0BE14DF60420854206D0B5F57F4F27
:1023100003D04FF60170854202D14FF0130BFDE060
:102320004FF0310BFAE0B8F1030F61D18149B1F8F8
:1023300040000421FEF7AFFD18B14DF604208542A0
:1023400014D07C49B1F840000421FEF7A4FD10B17F
:10235000B5F57F4F0AD07749B1F840000421FEF768
:102360009AFD78B34FF60170854230D1714890F8EC
:10237000200040B3A5F55A40043830B1A0F5105004
:10238000FC3850B101281BD100E000BF02273046C5
:10239000711C8EB20DF8007013E067488079022836
:1023A00001D1022706E064488079012801D1032782
:1023B00000E005273046711C8EB20DF8007000E079
:1023C00000BFABE003E0FFE74FF0330BA6E04DF6B4
:1023D0000420854206D0B5F57F4F03D04FF601703B
:1023E000854202D14FF0130B98E04FF0310B95E08E
:1023F000B8F1020F72D14F49B1F840000421FEF745
:102400004AFD18B14DF60420854214D04949B1F86F
:1024100040000421FEF73FFD10B1B5F57F4F0AD013
:102420004449B1F840000421FEF735FD78B34FF67A
:102430000170854258D13F4890F8200040B3A5F57F
:102440005A40043830B1A0F51050FC3808B30128C8
:1024500045D128E03848C08A3749898A884210D156
:102460003548C06939490840B0F1005F09D10422FC
:1024700031491C313148FFF70AFD08B9012700E056
:1024800002273046711C8EB20DF8007028E02BE058
:1024900027E000202849487104273046711C8EB27D
:1024A0000DF800701CE02448C0682549096888427E
:1024B0000BD02148006923490968884205D01E488D
:1024C000C08A21490988884201D1012700E00227FA
:1024D0003046711C8EB20DF8007001E015E000BFAF
:1024E0001CE04FF0330B19E04DF60420854206D076
:1024F000B5F57F4F03D04FF60170854202D14FF002
:10250000130B0BE04FF0310B08E00A48007901286B
:1025100004D10020074908714FF0120BAAF800609F
:10252000BBF1000F04D1324669464846FDF73CFE38
:10253000584623E6141F0020E01600200080000803
:102540008000002084000020880000200000FE2F72
:102550002DE9F04704460F4690469946002500268F
:1025600026782648D0F82C182548B0F84000801E60
:1025700008442249C1F82C08FEF748FC08B192250E
:1025800039E0FEF74DFC08B1932534E01C48B0F863
:10259000400040F60201884201DD13252BE0174878
:1025A00090F83008012806D0144890F83008022826
:1025B00001D024251FE0114890F82908B04201D02D
:1025C000732518E00D48D0F82C080E490968884298
:1025D00001D971250FE0012008494870022081F8D7
:1025E00030080748B0F84000821E074903482430ED
:1025F000FDF7DAFD78252846BDE8F087E0160020D3
:10260000141F0020440100208608002003480449CC
:102610000880000C091D088070470000345900082C
:10262000B86C004010B500F001F810BD0CB50020EA
:10263000019000904048006840F480303E490860B6
:1026400000BF3D48006800F4003000900198401C35
:102650000190009820B94FF6FF7101988842F0D19F
:102660003548006800F4003010B10120009001E00E
:1026700000200090009801285CD13048006840F0AC
:1026800010002E4908600846006820F0030008602A
:102690000846006840F00200086027484068264964
:1026A00048600846406848600846406840F48060DA
:1026B00048600846C06A224908401F49C862084667
:1026C000C06A204908431C49C8620846006840F0B7
:1026D0008060086000BF1848006800F000600028B3
:1026E000F9D01548406820F47C101349486008462A
:1026F000406840F4E81048600846006840F0807088
:10270000086000BF0C48006800F000700028F9D095
:102710000948406820F003000749486008464068BF
:1027200040F00200486000BF0348406800F00C0021
:102730000828F9D10CBD0000001002400020024022
:1027400000F0FEFF140801000F480068401C0E490D
:1027500008600E480068401C0C4908600A48006880
:102760004FF47A71B0FBF1F201FB1200012804D1A1
:1027700007480068401C064908600648007810B900
:102780000120044908707047340000202C0000200C
:10279000380000203000002030B5164800684FF4A3
:1027A0007A72B0FBF2F1B1F1807F01D301201DE01C
:1027B00021F07F40401E4FF0E022506150170F2261
:1027C000002807DA13071D0E0B4B00F00F04241F1F
:1027D0001D5503E013071C0E084B1C5400BF0020BE
:1027E0004FF0E022906107201061002008B100BF87
:1027F000FEE730BD0000002018ED00E000E400E03E
:1028000010B51648006840F00100144908600846F9
:10281000406813490840114948600846006811495A
:1028200008400E4908600846006820F480200860CF
:102830000846406820F4FE0048600846006820F022
:10284000A05008604FF47F0088600020C862FFF746
:10285000E9FE4FF000600449086010BD001002401E
:102860000000FFF0FFFFF6FE08ED00E010B50121CB
:10287000084800F016F858B10121064800F00EF89B
:102880000548006808B9012000E0002002490860FE
:1028900010BD00000004004090012342CA430282A0
:1028A000704730B50246002000230024158A05EA4F
:1028B0000103958905EA010413B10CB1012000E080
:1028C000002030BD10B51248008888B90020114999
:1028D00008701149087011490870114908701149B0
:1028E00008700846017810480088FEF705FF0DE0E3
:1028F0000720094908700D480078401C0B490870F2
:1029000008460078102801D10020087010BD000092
:10291000A6000020C2000020B00000209900002086
:10292000BE000020B70000209E0000209C00002078
:1029300010B5012021490870002021490870214864
:102940000078012805D120480078102801D1FEF731
:10295000A7FE1C480078012803D11B4800781028E6
:1029600005D01A48007858B11948007840B9962027
:10297000184908800120184908700220174908707A
:1029800016480078012802D11548007848B10E4851
:10299000007830B10B480078042804D11148008831
:1029A00008B900F0F9FC10480078012805D1054865
:1029B0000078062801D100F0EFFC10BDBA0000201D
:1029C000BF000020B0000020940000208C000020F8
:1029D0008B000020AC000020C10000208A000020F5
:1029E0008D000020920000209900002070B536482C
:1029F0000078012866D035480079012804D1344890
:102A00000078012800D170BDFEF7A8FE314908808A
:102A10003148FEF75FFE3048007800F0F0002F49A3
:102A2000087000202E4908802E4800882749A1F808
:102A30004000002008712848007800F00F05224867
:102A40000078022803D115B901201F4908702048D9
:102A50000078012801D100F09FFC2048007820BBBD
:102A60001D48007800F00F001E49088001240CE08A
:102A70001948005D1C491A4A128888541848008871
:102A8000401C17490880601CC4B216480088844264
:102A9000EEDD00F03DFA48B90920144908700846F7
:102AA000017810480088FEF727FE0BE0012010494E
:102AB000087000200D490870084601780948008810
:102AC000FEF71AFE00BF9EE78A000020141F0020B8
:102AD00099000020A4000020C4000020A0000020D5
:102AE000A20000209E00002084080020B7000020E3
:102AF000B900002010B51F480078012824D001201B
:102B00001D490870FEF72AFE1C4908801C48FEF784
:102B1000E1FD1B48007800F00F04164800780228F9
:102B200003D114B901201349087016480078012810
:102B300001D100F031FC0020134908700120134935
:102B400008701349087114E00F480078401CC0B2A7
:102B50000D49087002280CDB02F002FA00F064F85C
:102B6000002009490870034908700A4908700A4999
:102B7000087010BD8A000020BB000020A4000020C7
:102B8000C400002099000020CD000020CC000020CF
:102B9000141F0020B00000203801002010B511489B
:102BA000007838B1104840781049087000F0E6FB12
:102BB0000F4908700D4800780E4908700C480078DD
:102BC0000D49087000200D49087000F025FC0B48E5
:102BD000007818B904200A49087002E00320084967
:102BE000087010BDC3000020C40000208C0000202D
:102BF0008D0000208B0000208E000020900000201F
:102C0000B0000020004870478408002010B5054837
:102C10000078012804D100200249087000F050F922
:102C200010BD0000BB00002000200D4908700D49B8
:102C300008700D4908700D4908700D4908700D495C
:102C400008700D4908700D4908700D4908700D494C
:102C500008700D4908700D4908700D4908707047DB
:102C6000B00000208A00002099000020BD00002054
:102C7000BE000020BA000020BB000020BF000020E2
:102C8000C0000020C1000020C2000020B6000020CB
:102C9000BC00002010B507480078FEF78BFD064801
:102CA000FEF762FD462005490880012004490870AE
:102CB00010BD000098000020C4000020A8000020E3
:102CC000BF00002010B50446114804800088072882
:102CD00003DC00200F49087002E010200D49087045
:102CE00001200D49087000200C4908800C4800782C
:102CF000012802D100F04EFC09E00C2009490870BF
:102D000008460078FEF720FD00200349087010BD3A
:102D100092000020940000208A00002096000020ED
:102D2000BD000020B700002010B500F037FE00F015
:102D300033FB10BD10B50A48007820B1012805D03A
:102D4000022809D105E000F08DFA06E000F0A6FAAD
:102D500003E000F0D9FA00E000BF00BF10BD0000A2
:102D60009D00002010B52E4840782D49097801F0CB
:102D70000F0140EA01202B490880084600882A49B3
:102D800008802848008840F60201884213DD0D20A3
:102D9000264908700846017822480088FEF7ACFCF6
:102DA00002202349087000F07FFB002020490870B2
:102DB0002049087032E01B48008808282EDB00F00C
:102DC000A7F848B90920194908700846017815483C
:102DD0000088FEF791FC21E0022411E01048005D1C
:102DE0001549164A128888540F480088401E0E491B
:102DF000088012480088401C10490880601CC4B23A
:102E0000072CEBDD01200E49087006480088FEF70C
:102E100048FC01200B49087000F046FB10BD000083
:102E2000C40000209E000020A6000020B700002063
:102E3000B6000020B000002084080020A20000207E
:102E40009C0000209900002010B51848007800F080
:102E50000F001749088001240CE01448005D154953
:102E6000154A1288885414480088401C124908806A
:102E7000601CC4B20E4800888442EEDD00F048F8C1
:102E800048B909200D4908700846017808480088AB
:102E9000FEF732FC08E00020084908700846017877
:102EA00003480088FEF728FC10BD0000C400002085
:102EB0009E00002084080020A2000020B70000200F
:102EC00010B50E48007800F0F0000D4908700020A1
:102ED0000C4908800C490870094800780B4948766D
:102EE0000748007810B9FFF7AFFF05E00448007805
:102EF000102801D1FFF736FF10BD0000C4000020EC
:102F0000A0000020A2000020B9000020141F002013
:102F100000202149097831B1102912D0202918D078
:102F2000302935D12CE01D49098849B11C490A884E
:102F30001A490988491C8A4201DA002000E0012070
:102F400027E017490988082901DA002000E001205C
:102F50001FE014490988072907DB11490988082956
:102F600001DA00200BE0012009E00D490A880D4933
:102F70000988491C8A4201DA002000E0012008E0AB
:102F800007490988032901DA002000E0012000E058
:102F900000BF00BF70470000A00000209E0000207E
:102FA000A4000020A60000202B490988072932DA56
:102FB00001212A4A1180012016E02949095C294A89
:102FC000294B1B88D15428490988491C264A11805D
:102FD00026490988491E254A118020490988491C2B
:102FE0001E4A1180411CC8B21B4909888842E4DD91
:102FF0001E49098811B901211D4AD17701211D4AB5
:10300000117008211C4A117001211C4A1170002105
:10301000154A11801FE01049098807291BDB012090
:1030200011E00F49095C0F4A0F4B1B88D1540E4920
:103030000988491C0C4A11800C490988491E0B4A11
:103040001180411CC8B20728EBDD0849098811B975
:103050000121074AD1777047B2000020B400002058
:10306000C400002084080020A2000020A600002048
:10307000141F00209D000020B0000020BE00002092
:1030800010B52D48008838B903202C49087008462F
:10309000007800F0CFF84EE02948007801284AD1A6
:1030A000002027490870274908702748007800F059
:1030B000F000264908700846007818B108460078E4
:1030C000102809D106201D4908700846007800F034
:1030D000B1F8FFF7F5FE2EE01C48007820282AD131
:1030E000FFF716FF38B90920144908700846007820
:1030F00000F0A0F81FE01448007800F00F00144919
:103100000978884210D1002012490870FFF712FE9A
:1031100096200949088001200A4908700D48007866
:1031200048B9FFF7CFFB06E00420044908700846C1
:10313000007800F07FF810BDAE000020B70000203E
:10314000BB000020C2000020C4000020A00000201E
:103150009C0000209D00002010B52C4A12882C4BAA
:103160001B889A421FDB2A4A1178012011E0294A64
:10317000125C294B294C24881A55284A1288521C63
:10318000264B1A80224A1288521E214B1A80421C5A
:10319000D0B28842EBDD1E4A1288002A35D10122C6
:1031A0001F4BDA7731E0194A1288194B1B889A4273
:1031B0002BDA01221B4B1A80012016E0154A125C03
:1031C000154B164C24881A55144A1288521C134B5E
:1031D0001A800F4A1288521E0D4B1A80114A12880B
:1031E000521C104B1A80421CD0B2084A12889042DE
:1031F000E4DD02220C4B1A7008220C4B1A700122DB
:103200000B4B1A700022054B1A8010BDB200002033
:10321000A6000020C400002084080020A200002096
:10322000141F0020B40000209D000020B0000020EA
:10323000BE00002010B50446214606480088FEF76F
:103240005BFA0020044908700449087004490870BA
:1032500010BD00009E000020B0000020990000205A
:10326000BE00002010B50A48008840F60201081A86
:103270000849088008480088072802DBFFF794FE09
:1032800005E005480088072801DAFFF765FF10BD53
:10329000A2000020B2000020A60000201248007802
:1032A00008BB16E0114812490988405C1149124ACE
:1032B0001288885410480088401C0F4908800F4825
:1032C0000088401E0D49088009480088401C0849B4
:1032D0000880074800880728E4DD002008490870B6
:1032E0000720084908707047BE000020C400002075
:1032F000B400002084080020A2000020A6000020C6
:103300009D000020B00000201449097821BB144919
:10331000087816E01349144A1288895C134A144B42
:103320001B88D15412490988491C114A11800C4943
:103330000988491E0A4A11800B490988491C0A4A12
:10334000118009490A88411C8A42E3DD0021094AAB
:1033500011700721084A117070470000BE0000205C
:10336000A6000020C4000020B40000208408002033
:10337000A20000209D000020B0000020054A9178A6
:1033800031B17F2900DD7F21C8B2421CD0B200E0FC
:1033900001207047C400002010B5144800780928A7
:1033A00021D2DFE800F005080B0E1114171A1D00DA
:1033B000FFF72CFC18E000F069FC15E000F0D4FBEE
:1033C00012E000F01BF80FE000F02EFB0CE000F024
:1033D00097FC09E000F02CFC06E0FFF751FE03E04B
:1033E00000F096FB00E000BF00BF10BDB000002061
:1033F0000120014908707047BD00002010B500F0A1
:103400000BF80348007810B904200249087010BD79
:1034100090000020B000002010B50A48007820B1CC
:10342000012805D0022809D105E000F0C9F906E01D
:1034300000F0ECF903E000F02BFA00E000BF00BF61
:1034400010BD00009000002012490988C1F303213B
:1034500041F01001104A11700E4909785170022094
:1034600011E00E490E4A1288895C0B4A11540C492E
:103470000988491C0A4A118006490988491E054ADB
:103480001180411CC8B20728EBDD0821054A1170E4
:103490007047000092000020C40000208408002033
:1034A000960000209800002010B51748007840F0E2
:1034B0003000164908700020487088701449088050
:1034C000032014490870032404E000200F49085524
:1034D000601CC4B2072CF8DD08200E4908700020DB
:1034E000FEF76EF90B480078FEF764F90748FEF71F
:1034F0003BF9062008490870462008490880012049
:103500000749087010BD0000B6000020C40000206C
:103510009A00002098000020B0000020AA0000209F
:10352000C0000020164A1278164B1A7001200121A3
:103530000EE0154A154B1B88D25C124B5A54134AA5
:103540001288521C114B1A80421CD0B24A1CD1B2B4
:103550000B4A12889142ECDD094A1278521C0C4B3E
:103560001A7007280ADC04E00022064B1A54421C99
:10357000D0B20728F8DD0822054B1A70704700000A
:1035800092000020C4000020840800209600002043
:103590009800002010B51048007810B9FFF7C2FF5E
:1035A00005E00D480078102801D1FFF74DFF0120FC
:1035B0000A4908700A480078FEF7FCF80948FEF747
:1035C000D3F80120084908704620084908800120E6
:1035D0000749087010BD0000940000208F000020F3
:1035E00098000020C4000020B0000020A8000020A7
:1035F000BF00002010B52A48008807282BDA0120D8
:1036000028490880012416E0274828490988405C99
:103610002749085525480088401C2449088025482A
:103620000088401E234908801E480088401C1D4910
:103630000880601CC4B21A4800888442E4DD01207E
:103640001D49087000201D490870FEF7C7F80020CA
:103650001649088023E01248008807281FDB012450
:1036600011E0114811490988405C114908550F487B
:103670000088401C0D4908800E480088401E0D49F6
:103680000880601CC4B2072CEBDD08200C490870D0
:10369000FFF700FB04200B49087000F065F910BD2E
:1036A000B2000020B4000020840800209600002012
:1036B000C40000209200002090000020BD000020E7
:1036C00098000020B000002070B5334800883349CE
:1036D000098888422DDB012530480678012413E053
:1036E0002F4830490988405C2F4908552D480088EB
:1036F000401C2C49088029480088401E2749088022
:10370000681CC5B2601CC4B2B442E9DD274806702B
:1037100004E0002024494855681CC5B2072DF8DD97
:10372000082022490870FFF7B5FA042020490870E4
:1037300030E0194800881949098888422ADA0120AE
:103740001C490880012416E0154816490988405C88
:103750001549085513480088401C124908800F4835
:103760000088401E0D49088012480088401C1149FD
:103770000880601CC4B2084800888442E4DD02204E
:103780000D49087000200D490870FEF727F8002049
:103790000449088070BD0000B200002092000020A3
:1037A0008408002096000020C4000020980000201B
:1037B000B0000020B400002090000020BD000020D8
:1037C00010B50D48007840F020000C4908700C48F6
:1037D000008840F60201081A0A4908800A48008851
:1037E000072802DBFFF706FF05E0074800880728E7
:1037F00001DAFFF769FF10BD8F000020C400002030
:1038000096000020B20000209200002010B517485A
:103810000078012828D116E0154816490988405C2F
:103820001549164A1288885412480088401C1149CC
:10383000088013480088401E114908800F480088FE
:10384000401C0E4908800D4800880728E4DD082048
:103850000C490870FFF71EFA00200B49087004207D
:103860000A49087000F080F810BD0000BD0000207B
:103870008408002096000020C4000020B40000202E
:10388000920000209800002090000020B00000204E
:1038900010B52048007801283AD11F4804780078F4
:1038A0001E49097808441E49087018E01D481E4941
:1038B0000988405C1D49184A128888541A480088B3
:1038C000401C1949088015480088401E134908808B
:1038D000601CC4B210480088401C0F4908800E4884
:1038E00000880F4909788842E0DB04E000200F4996
:1038F0000855601CC4B2072CF8DD08200849087080
:10390000FFF7C8F900200A49087004200949087027
:1039100010BD0000BD000020B40000209200002077
:10392000980000208408002096000020C400002099
:1039300090000020B000002010B504462046FDF79E
:1039400003FF002004490870044908700449087006
:103950000449087010BD0000B00000208A0000205B
:10396000BD000020BA00002009480078401C08492A
:10397000087008460078102801D10020087005481A
:10398000007820B104480078401E03490870704751
:103990008F0000208C0000208B0000201A48007847
:1039A000012808D119480088002804DD174800883C
:1039B000401E1649088016480078012808D115488D
:1039C0000088002804DD13480088401E1149088043
:1039D00011480078012808D110480088002804DD2B
:1039E0000E480088401E0D4908800D4800780128C7
:1039F00008D10C480088002804DD0A480088401ED1
:103A00000849088070470000BF000020A80000207F
:103A1000C0000020AA000020C1000020AC0000204F
:103A2000C2000020AE00002010B52C48008838B934
:103A300001202B49087008460078FFF77DFF4CE015
:103A400028480078012803D027480078012844D16D
:103A5000002026490870234908702548008838B995
:103A600000201F49087008460078FFF765FF34E022
:103A70002048007848B12048007830B900201F491C
:103A8000087002201E49087027E01E48007818B10F
:103A90001C48007801280CD1FFF7BEFC1A480078BA
:103AA00018B900201049087017E001200E4908706D
:103AB00013E014480078022803D10320104908704D
:103AC0000BE010480078022807DD10480078401EFF
:103AD0000E49087005200A49087010BDA800002092
:103AE000B7000020BA000020BC000020BF0000206A
:103AF000920000208C0000208B000020C3000020DA
:103B0000B00000208D000020900000208E000020DA
:103B100010B51148008838B90320104908700846CC
:103B20000078FFF787FB15E00D48007801280AD1DF
:103B300000200B4908700B200849087008460078DF
:103B4000FFF778FB06E0FFF7F5F80648007808B9BC
:103B5000FEF7B8FE10BD0000AE000020B700002048
:103B6000BB0000209D00002010B52B48008838B90C
:103B700002202A49087008460078FFF7DDFE49E078
:103B800027480078012845D100202549087025489C
:103B9000007800F0F00024490870084600783028CA
:103BA00038D10020214908701E48007800F00F0429
:103BB000FFF7AEF938B909201849087008460078AF
:103BC000FFF7BAFE26E0032C07DB05201349087037
:103BD00008460078FFF7B0FE1CE0022C07D1082051
:103BE0000E49087008460078FFF7A6FE12E0012C87
:103BF0000DD107200949087008460078FFF79CFEA0
:103C000095200549088001200849087002E00CB998
:103C1000FEF7C4FF10BD0000AC000020B70000207C
:103C2000BB000020C4000020A0000020C100002034
:103C300010B50F48007801280ED100200C490870FB
:103C40000C49087007200C49087096200B49088021
:103C500001200B49087009E00A48008830B90120AA
:103C60000949087008460078FFF7E4FA10BD000023
:103C7000BA000020C0000020B0000020AE000020EC
:103C8000C2000020AA000020B700002010B515488F
:103C9000008838B901201449087008460078FFF7F9
:103CA0004BFE1DE011480078012819D100200F4972
:103CB00008700F4908700F48007838B900200A4989
:103CC000087008460078FFF737FE09E009480078D9
:103CD000102805D101200849087002200749087002
:103CE00010BD0000A8000020B7000020BA0000208E
:103CF000BF00002094000020C3000020B00000207E
:103D000008480078401E07490870084600780128D6
:103D100006DC032004490870044800780149087053
:103D2000704700008E000020B00000208D000020B1
:103D30000246002321B90D48006810600120704739
:103D40000A4803681068984205D81068181A884213
:103D500009D30120F3E71068C0F1FF30184488420E
:103D600001D30120EBE70020E9E700003400002048
:103D70004F48007801280AD14E484089401C4D49DF
:103D800048810120087000204949087000E0704710
:103D900048484089052190FBF1F201FB120030B93F
:103DA0004448408918B101204249487000E0EEE7DC
:103DB000404840890A2190FBF1F201FB120028B92A
:103DC0003C48408910B101203A49887039484089FF
:103DD000142190FBF1F201FB120028B9354840890B
:103DE00010B101203349C87032484089322190FB1C
:103DF000F1F201FB120028B92E48408910B10120D0
:103E00002C4908712B484089642190FBF1F201FB99
:103E1000120028B92748408910B10120254948716E
:103E2000244840894FF4FA7190FBF1F201FB120033
:103E300028B92048408910B101201E4988711D48C9
:103E400040894FF47A7190FBF1F201FB120028B91E
:103E50001848408910B101201649C8711548408999
:103E600040F2DC5190FBF1F201FB120028B911483D
:103E7000408910B101200F4908720E4840894FF463
:103E8000FA6190FBF1F201FB120028B90948408960
:103E900010B10120074948720648408941F270710B
:103EA000884202DB00200349488100BF6FE7000021
:103EB00030000020900100200FB51848007832280B
:103EC00002DB00201549087014480278001D00EB41
:103ED0000210009901609DF8041010480278001D3E
:103EE00000EB021001719DF80D100C480278001DC6
:103EF00000EB0210417309480178001D00EB01102E
:103F0000DDF8051040F8051FDDF809104160034891
:103F10000078401C014908700FBD00008810002087
:103F200010B51748006800B110BDFCF74BFF00B991
:103F3000FAE71BE013484078322802DB00201149E1
:103F4000487010484178001D00EB011494E80F0000
:103F500001F097F901200C498870002081F82800B1
:103F600008484078401C0749487005E0054800783B
:103F7000044949788842DDD100BF00BFD4E7000082
:103F80006800002088100020141F002010B5094888
:103F9000807E70B10748407F10280AD10549087F0C
:103FA00000F05CFB002003498876FF210248FCF703
:103FB00022F910BD141F00208408002010B5074806
:103FC000807E50B10548407F112806D10348293032
:103FD00000F00EFC00200149887610BD141F00205F
:103FE00010B50648807E40B10448407F222804D1A5
:103FF00000F074FA00200149887610BD141F0020DB
:1040000010B51448807E20B31248407F272820D165
:10401000104890F82900062809D00F4A0D49293187
:10402000052000F045FC00200A49887611E0094887
:1040300090F8290006280CD1074A0649293100F0DA
:1040400037FC002003498876C877034800210160C7
:10405000416010BD141F0020EC00002010B50A487C
:10406000807E78B10848407F28280BD1022106487D
:10407000293000F03BFD002003498876FF210348EA
:10408000FCF7B9F810BD0000141F002084080020C0
:1040900010B50948807E70B10748407F2E280AD1AC
:1040A00006480088401E81B2054800F05DFA0020F5
:1040B0000149C877887610BD141F0020A200002097
:1040C0008508002010B50A48807E78B10848407FF6
:1040D00031280BD103210648293000F091FD002042
:1040E00003498876FF210348FCF785F810BD0000DE
:1040F000141F00208408002010B50C48807E98B161
:104100000A48407F34280FD109480088401E81B2F8
:10411000084800F0AFFD0020044988764877FF2169
:104120000448401EFCF767F810BD0000141F002073
:10413000A20000208508002010B50C48807EA0B1A8
:104140000A48407F362810D109480078401EC1B285
:104150000648293000F01CFE002004498876487784
:1041600040F602010348FCF746F810BD141F00207A
:10417000A20000208408002010B50948807E70B19C
:104180000748407F37280AD106480088401E81B280
:10419000054800F027FE002001498876487710BDC9
:1041A000141F0020A20000208508002010B5074839
:1041B000807E50B10548407F3E2806D10348293013
:1041C00000F012FA00200149887610BD141F00206B
:1041D00010B50A48807E78B10848407F85280BD109
:1041E00001210648293000F055FE00200349887659
:1041F000FF210348FBF7FFFF10BD0000141F002044
:10420000840800208178064A1170C17851701146E7
:104210000978491C117011464978891C5170704702
:10422000EC00002010B50948007801280DD107489E
:1042300040780D2806DA05484078054951F82040B5
:10424000A04702E000200149087010BDF4000020E2
:10425000F800002010B501200249087000F080FE2F
:1042600010BD0000F400002010B5002002490870C5
:1042700000F076FE10BD0000F40000202DE9F041B2
:1042800000240125A046002600277E48007801284A
:104290001DD100207B4908700846407988B901206B
:1042A00048710846C06878490860764800697749CF
:1042B0000860002076490860764908807149887155
:1042C000DDE003206F49887100204871D7E06D4818
:1042D0004079012869D16B4988716C48006890B1B8
:1042E0006A480068B0F5006F08D968480068A0F512
:1042F0000060664908604FF4006704E0634807689F
:1043000000206249086060490968614A126888189B
:104310003946FCF78CFE05465D48006838445C4928
:1043200008605C480088401C5A4908802DB1032071
:104330005449887100204871A1E05448006830BB9E
:104340000220504988710020487171222046611C6A
:10435000CCB251490A5401222046611CCCB24E49CC
:104360000A54FF222046611CCCB24B490A54002259
:104370002046611CCCB248490A5401222046611CE7
:10438000CCB245490A542046FDF748FA77E0414847
:104390000088142190FBF1F201FB120000286ED17D
:1043A00078213120FDF71CFA69E036484078012871
:1043B00065D176222046611CCCB237490A54314877
:1043C00090F829282046611CCCB233490A5433485E
:1043D000B0F84000861E32462A492431081FFCF7F7
:1043E000B3FC28488068A0B926481630FCF760FC6A
:1043F000042224492431A1F10E00FCF75DFC214880
:10440000406A2049C861FF2204211E482430FBF77E
:10441000EBFE1C498968224A881832461949243122
:10442000FDF735FD0546174880683044154988601A
:104430000846D0F82C081B490968884209D3194856
:104440000068061F32461649091D0E481630FCF753
:1044500033FC25B910492046FDF7E0F906E00020BD
:104460000849C86172213620FDF7BAF9054890F86D
:104470002908401C034981F8290800204870BDE83C
:10448000F0810000E01600205001002054010020BF
:10449000580100205C01002068210020141F00202A
:1044A00000800008440100200A200B4981F8270001
:1044B0000120C870002081F826000120C876002065
:1044C00081F820008871C88781F8220081F82300D4
:1044D00081F8250070470000141F002070B50024EB
:1044E00000251E484078012837DD1D480079012845
:1044F00033D11B48B0F84000032824DB1849B1F839
:10450000400000EBD0714910A0EB4101012918D106
:104510001349B1F84010032913DC1248FCF766FF79
:104520000546032D04DB0F492846FDF777F90BE01C
:104530000B48B0F84C0040F27771884204D1312426
:1045400002E0132400E013241CB121462220FDF7D1
:1045500047F91E200249A1F8440070BD480100201F
:10456000141F0020682100202DE9F04104460D466B
:10457000002600271948407801282CDD18480079CA
:10458000012828D11649C87E00220221FCF752FCDE
:10459000B8B1032D01DA132714E0A81E81B220461A
:1045A000FDF792FD064656B96E200E490870207838
:1045B0004870607888700320FDF730F902E03746D4
:1045C00000E07F271FB139462E20FDF709F928208A
:1045D0000349A1F84400BDE8F08100004801002033
:1045E000141F00206821002070B504460025002615
:1045F0001748407801282ADD1649B1F84000022109
:10460000FCF749FCC8B1207800F07F0666B9207835
:10461000FCF73AFC90B17E200F4908702078487072
:104620000220FDF7FBF809E00A480079012805D1CE
:10463000002008490871122500E013251DB1294604
:104640003E20FDF7CDF80A200249A1F8440070BDD4
:1046500048010020141F0020682100202DE9F041AE
:1046600005460227002600245D48407801287CDDAD
:1046700010205B490870002048705A49B1F840008A
:104680000221FCF708FC002870D005F07F04012C03
:1046900003D0022C01D0032C69D15248C07E0328DC
:1046A0003AD1022C38D1FCF7FDFB002832D04D481E
:1046B000C476C47600204B4981F820008871C887F1
:1046C00081F8220081F8230081F825002846FCF7B4
:1046D000DBFB80B15020444908700846457000203B
:1046E00088703220C87001200871F42048710627B4
:1046F0003846FDF793F800203C4981F8240881F8FA
:10470000250881F8260881F8280881F8270881F80B
:10471000300856E0222654E03248C07E012801D1FC
:10472000022C05D02F48C07E022803D1032C01D1D2
:10473000222646E0FCF7B6FBB0B3032C03D10020E1
:104740002849C87300E000BF2648C47600202549E8
:10475000C88781F8200088710846C07E032801D1EF
:10476000032C0BD000201F4902E037E028E01EE0B8
:1047700081F8220081F8230081F825002846FCF703
:1047800083FBF0B15020184908700846457000209E
:1047900088703220C87001200871F4204871062703
:1047A0003846FDF73BF80CE0FFE7222609E00D480C
:1047B0000079012805D100200A490871122600E07D
:1047C00013261EB131461020FDF70AF80A200449CD
:1047D0008880084680880349A1F84400BDE8F0813C
:1047E00048010020141F002068210020E01600204E
:1047F00070B50446002500262948407801284DDD83
:10480000112027490870002048701E208880254804
:104810000079012842D12349B1F840000221FCF778
:104820003AFB002830D0207800F07F063046FCF7B5
:1048300023FB00B3FCF736FBD8B12078FCF724FB50
:1048400038B1512018490870207848700220FCF7D0
:10485000E5FF16480079012805D1002013490871A9
:1048600011490870487001200E490870C8208877E7
:104870000BE0222509E00B480079012805D1002032
:1048800008490871122500E013251DB129461120A1
:10489000FCF7A6FF0A200349A1F8440070BD000000
:1048A00048010020141F002068210020E01600208D
:1048B0002DE9F04781460C46154600274FF0FF08CA
:1048C00084484078012876DD83480079012872D138
:1048D0008149C87E01221146FCF7ACFA00286BD052
:1048E0002078032843D100207C4908707A49B1F828
:1048F00040000221FCF7CFFA002836D07648C07875
:10490000012801D13727D7E0FCF7CCFA08B92227D4
:10491000D2E0672072490870207848707148FCF72F
:104920005AFD8046B8F1000FEDD16B4890F8200099
:10493000012807D168488079012803D168480021FF
:10494000418003E066486749098841800120634946
:1049500008706149887167205E49087000204870BE
:104960005F490420FCF75AFFA6E01327A4E0207853
:1049700004287DD15849B1F840000421FCF78BFA96
:10498000002876D0FCF78EFA08B9222794E0524826
:1049900090F82600022802DC5048007868B94E489A
:1049A00090F82600032800DB36274C4800780028C2
:1049B000A9D1242780E08AE07DE0484800780128DA
:1049C00002D10020454908704548002101600222BB
:1049D0004449FBF71BFC00285DD042494978414A15
:1049E000127801EB022188B2FCF7C4FC064660781D
:1049F0002870A0786870E078A8702079E87030128C
:104A0000394908704E7002222846FBF7FFFBF8B9BF
:104A10000020314981F8260067203149087020784C
:104A200048702078062801D1012000E002202A49A0
:104A300081F8210067202749087000204870012074
:104A4000254981F8200026490220FCF7E7FE23E0F3
:104A5000214890F82600FF2806DA1F4890F8260023
:104A6000401C1D4981F826001B4890F8260001E0F3
:104A700018E015E0012801DC35270DE0164890F814
:104A80002600022808D136270A20134981F827007A
:104A90000120C87000E024271248002101600BE0CB
:104AA000132709E00C48B0F84000022801DA132768
:104AB00002E0122700E07F271FB139462720FCF7CC
:104AC0008FFE1E20034988800349A1F84400BDE8F9
:104AD000F087000048010020141F00205E01002024
:104AE00068210020780000207A0000202DE9F041A4
:104AF0000446884600270025002668203D490870A6
:104B00003D484078012873DD28203B4908701E206D
:104B100088803A49C87E01221146FCF78BF90028AB
:104B200055D03649B1F840000321FCF7B4F900280C
:104B30004BD0FCF7B7F9002845D0207800F07F056E
:104B400066780DB1032D35D1012E01D0032E28D169
:104B50006DB9012E04D10020284981F8220015E00A
:104B60000020264981F8220081F823000EE0032D61
:104B70000CD1012E04D10120204981F8220005E04A
:104B800001201E4981F8220081F823002078FCF7DB
:104B90007BF920B32078174948700220FCF73EFECD
:104BA0001DE01648B0F84C0040F27771884216D1EB
:104BB000312714E011480079012810D100200F4955
:104BC000087112270BE0222709E0132707E00B48A2
:104BD000B0F84C0040F27771884200D17F271FB1B6
:104BE00039462820FCF7FCFD0A200449A1F84400BE
:104BF000BDE8F0816821002048010020141F00203A
:104C0000F8B505460E46002400200090164840786E
:104C1000012827DD3120144908701E2088801348A0
:104C2000007901281ED11149C87E01221146FCF7E6
:104C300001F938B16B460E4A31462846FDF78CFA29
:104C4000044600E07F2424B121463120FCF7C8FD52
:104C500004E00749BDF80000FCF7E0FD0A20034925
:104C6000A1F84400F8BD000048010020141F0020F6
:104C7000682100202DE9F04104460E4600273D48FA
:104C80004078012874DD3C48007908B9BDE8F0811E
:104C90003949C87E00220221FCF7CCF8002855D003
:104CA000354890F8200001284ED1257894F80180ED
:104CB0000A2E47D115B9B8F1440F01D0312746E08B
:104CC000A0780006E17840EA0140217940EA01201D
:104CD0006179084329490860A0790006E17940EA32
:104CE0000140217A40EA0120617A084324490860A2
:104CF0007420244908700846457020204870082018
:104D000088700220C87001201F4981F829080020FE
:104D1000C1F82C088860194800681C4988420FD1E6
:104D200017480068B0F5563F0AD2174890F8240893
:104D300020B114490420FCF771FD08E0222706E0A9
:104D4000702704E0132702E0332700E07F2727B114
:104D500039463420FCF744FD03E001200A4981F87C
:104D600030081E200349888014200349A1F844001C
:104D700000BF8BE748010020141F002040010020E5
:104D80004401002068210020E01600200080000877
:104D9000F8B505460E460024002000900E484078E5
:104DA000012818DD36200C4908701E2088800B4829
:104DB000007901280FD16B46094A31462846FDF794
:104DC000C7FB04461CB121463620FCF709FD1E2016
:104DD0000249A1F84400F8BD48010020141F00203A
:104DE0006821002070B505460E460024772025492D
:104DF000087025484078012843DD244800790128BF
:104E00003FD17720204908701E20888000204870FC
:104E10001E49C87E00220221FCF70CF838B31B485B
:104E200090F82000012820D11849B1F84000012154
:104E3000FCF731F8B8B1164890F83008022810D1C4
:104E4000772010490870124890F82000C04348703D
:104E500003200F4981F830080A490220FCF7DEFCE4
:104E600006E0242404E0132402E0332400E07F243D
:104E70001CB121463720FCF7B3FC0A200349A1F8F6
:104E8000440070BD6821002048010020141F00204C
:104E9000E01600202DE9F04104460F4600260025CB
:104EA0002C484078012853DD85202A4908701E20AF
:104EB00088802949C87E01221146FBF7BBFF0028E4
:104EC00035D02549B1F840000221FBF7E4FF60B37B
:104ED000FBF7E8FF08B9222631E0207800F07F05D3
:104EE000012D01D0022D17D1012D04D100201A4926
:104EF00081F8250003E00120174981F8250020787A
:104F0000FBF7C2FFD8B1C52014490870207848705B
:104F10000220FCF783FC12E00F48007901280ED133
:104F200000200D490871122609E0132607E00A48FF
:104F3000B0F84C0040F27771884200D17F261EB154
:104F400031468520FCF74CFC0A200349A1F84400B7
:104F5000BDE8F08148010020141F002068210020D6
:104F600010B5FCF7BBFA012823D102201649C876F8
:104F700001200873002081F820008871C88781F81B
:104F8000220081F8230081F8250081F82700C870ED
:104F900050200E4908700C48C07E48700020887070
:104FA0003220C87001200871F42048710620FCF7F7
:104FB00035FC0020064908700220487001208870E6
:104FC0000020888010BD0000141F002068210020F0
:104FD0004801002010B50848807E58B10649487F36
:104FE00000F014F80020044988764877FF21034830
:104FF000FBF701F910BD0000141F002084080020F9
:1050000010B50446FFF730F910BD000070B5054635
:10501000002415484078012825DD1448407F3428B5
:1050200007D01248407F362803D01048407F3728E9
:1050300008D10E49C87E00220221FBF7FBFE48B9C9
:105040007F2407E009480079012803D1002007499F
:10505000087111241CB121462846FCF7C1FB0A2027
:105060000249A1F8440070BD48010020141F00202F
:105070001E200149888070474801002070B5054610
:105080000C4605480078272805D16078012802D110
:105090002046FFF7B7F870BD480100202DE9F04128
:1050A00007460E4614464EBB3F484078012825D19E
:1050B0003D48007840302178884207D12146384663
:1050C000FFF7DCFF0220384948706BE020787F282A
:1050D00068D1354800786178884263D1A078782813
:1050E00005D1FFF7C5FF04202F4948705AE0A0788A
:1050F000FFF786FF03202C49487053E0002E44D16F
:1051000029484078022840D12078102805D1022073
:1051100025494870607825490877207823494877E1
:10512000002518E02248405D2049497F884210D17F
:105130001E48407F342803D01C48407F362805D1C4
:105140001C48008820B91C48457001E01A48457089
:1051500003E0681CC5B20D2DE4DB00BF0D2D02D1AC
:105160000C2015494870142110482930FBF743F8EA
:105170001422611C0D482930FBF716F801200B4959
:1051800088760846A0F840700CE0092E0AD10B483A
:105190000078012806D1002008490870FF2108483E
:1051A000FBF729F8BDE8F08148010020141F00201A
:1051B000FA5B0008A6000020F4000020CC000020CC
:1051C00084080020012001494870704748010020F0
:1051D000704710B500F098F810BD70B504460D4644
:1051E000164632462946204600F06EFA70BD70B56C
:1051F00004460D46164632462946204600F0A7FAD8
:1052000070BD00001149096851B94FF0E02189696A
:105210000E4A1160114609680D4A51430B4A11604C
:105220004FF0E0218969094A12688818074909681E
:1052300043F285621144054A116080B21146098823
:1052400001EB810140EA014070470000D0000020DE
:105250000DE37A050FB41FB5069800909DF8220063
:105260008DF804009DF804200DF123010DF10500D7
:10527000FAF79AFF9DE80F0000F0C4F81FBC5DF834
:1052800014FB0FB587B000208DF81000079802902E
:105290009DF820008DF8120000208DF811009DF877
:1052A00012200DF121010DF11300FAF77DFF069890
:1052B000009002A80FC8FBF753FD0BB000BD10B55E
:1052C0000A20FBF743FEFCF7A7FD10BD10B503480D
:1052D000027803A10B48FAF767FF10BD785B00085E
:1052E000515246424C5F312E305F323330333034CE
:1052F00020202020202020202020202020202020AE
:10530000000000003006002010B53748007850B982
:10531000FFF7DCFFFBF7DCFDFBF716FEFFF7C4F839
:1053200001203149087031480078D8B12F48807F7A
:1053300028B12E48807F401E2C49887711E000203C
:105340002A49087000BF2A48006800F4E060294933
:105350000843001D26490860BFF34F8F00BF00BF00
:10536000FEE710BD24480088401C80B22249088016
:1053700004280DDB00200880FEF76CFF01201B498C
:10538000C8710020487600F07BF800201B49088097
:105390001B480088401C80B219490880012819DB8D
:1053A00000200880FEF73EFFFCF7CAF90F48407E58
:1053B000102803D00D48407E20280BD10F480088CC
:1053C000401C80B20D490880012803DB00200880C2
:1053D00000F056F8FEF7A4FDFCF79EF8FBF7F6FC8C
:1053E000FEF74CFF00BFBCE7EA000020141F0020BE
:1053F0000CED00E00000FA05E4000020E8000020C9
:10540000E60000200FB540F2DF710098884204D01A
:1054100040F27771009888422ED1184800783228DF
:1054200002DB00201549087014480278001D00EBCB
:105430000210009901609DF8041010480278001DC8
:1054400000EB021001719DF80D100C480278001D50
:1054500000EB0210417309480178001D00EB0110B8
:10546000DDF8051040F8051FDDF80910416003481C
:105470000078401C014908700FBD0000AC130020EB
:1054800010B51DE012484078322802DB0020104998
:1054900048700F4840780F4908700D484178001D4A
:1054A00000EB011494E80F00FCF7C6FC08484078B4
:1054B000401C0749487008480068401C06490860BD
:1054C00003480078024949788842DBD110BD0000CA
:1054D000AC130020D5000020E000002000BFFEE754
:1054E00044E032213EE000BF00BF00BF00BF00BF6C
:1054F00000BF00BF00BF00BF00BF00BF00BF00BFB4
:1055000000BF00BF00BF00BF00BF00BF00BF00BFA3
:1055100000BF00BF00BF00BF00BF00BF00BF00BF93
:1055200000BF00BF00BF00BF00BF00BF00BF00BF83
:1055300000BF00BF00BF00BF00BF00BF00BF00BF73
:1055400000BF00BF00BF00BF00BF00BF00BF00BF63
:1055500000BF00BF00BF00BF00BF00BF00BF00BF53
:105560004A1ED1B20029BEDC421ED0B20028B8DCEF
:10557000704702E008C8121F08C1002AFAD170471C
:105580007047002001E001C1121F002AFBD17047C3
:1055900008B501210820FCF7BFFC03208DF80200AC
:1055A00014208DF803004FF48060ADF800006946C8
:1055B0000D48FBF708FE03208DF802004FF4006051
:1055C000ADF8000014208DF8030069460648FBF78B
:1055D000FAFD4FF480610448FBF7CAFE4FF4006106
:1055E0000148FBF7C5FE08BD000C0140022808DA9F
:1055F000074911F8301021B1054911F8301003297D
:1056000000D170470221024A02F8301000BFF8E7CB
:105610006C01002010B50446022C03DA0C4810F887
:10562000340000B910BD0320094901F8340001EB32
:10563000C401081D0021FEF77BFB1CB90548FAF7E1
:10564000DDFF02E00448FAF7D9FF00BFEAE70000F7
:105650006C0100200064004000680040022800DB6C
:1056600070470121024A02F8301000BFF8E700003D
:105670006C010020022803DA074911F8301001B943
:1056800070470121044A02F83010002102EBC002E9
:10569000517000BFF4E700006C01002001460229B0
:1056A00008DA064810F8310020B1044810F831003B
:1056B000032801D1002070470120FCE76C01002085
:1056C00010B5FFF765FF10BD2DE9F04107460C4608
:1056D0001646FCF759F9A020FCF728F9FCF782F9E7
:1056E00000B130E0A046E11704EB1161C1F30720DF
:1056F000FCF71CF9FCF776F900B124E0E0B2FCF706
:1057000015F9FCF76FF900B11DE0FCF73DF9A12098
:10571000FCF70CF9FCF766F900B114E000250BE08A
:10572000711EA94201D0012100E000210846FCF7CA
:10573000D3F87855681C85B2B542F1DBFCF73EF929
:105740000120BDE8F081FCF739F90020F9E72DE9E7
:10575000F04706460F4690463C46002534E035B1FA
:10576000E11704EBD1614911A4EB411109BB25B14B
:10577000FCF724F90620FBF7E9FBFCF705F9A0206C
:10578000FCF7D4F8FCF72EF900B124E0A146E117AC
:1057900004EB1161C1F30720FCF7C8F8FCF722F90C
:1057A00000B118E0E0B2FCF7C1F8FCF71BF900B15A
:1057B00011E0705DFCF7BAF8FCF714F900B10AE0EB
:1057C000601C84B2681C85B24545C8DBFCF7F6F85E
:1057D0000120BDE8F087FCF7F1F80020F9E7002090
:1057E00001E0411C88B23C28FBDB704786B0FDF726
:1057F00007F8FAF756FDFCF7D1F9FCF7CDFF01A841
:10580000FCF79AFBFCF7BFFAFCF7FAF9FFF758FF31
:10581000FCF728F9FAF792FD4FF400712648FBF7E0
:10582000A5FDFFF74CFDFBF765FE43E0FEF7A0FA90
:1058300022480078012805D1002020490870FFF790
:10584000C8FC37E01D484078012805D100201B49DD
:105850004870FCF703F92DE018488078012805D13D
:10586000002016498870FFF7B3FC23E01348C07886
:10587000012803D100201149C8701BE00F480079AE
:10588000012803D100200D49087113E00B4840792D
:10589000012803D10020094948710BE00748C0796D
:1058A000012807D100200549C8714FF40071024852
:1058B000FBF75CFDBAE70000000C014090010020FE
:1058C0002DE9F04704460F46154699463DB161194A
:1058D0000E48814203D8A0F50070844203D24FF0F5
:1058E000FF30BDE8F08737B1002602E0B85DA05573
:1058F000761CAE42FAD30648A4EB0008AAB21FFAFF
:1059000088F12046FFF773FC0020EAE768210020B9
:10591000681F00202DE9F04104460D4616461F463B
:105920003B46324629462046FFF7CAFF804640469E
:10593000BDE8F081515246424C5F312E305F323328
:105940003033303420202020202020202020202010
:1059500020202020000000002110422063308440DD
:10596000A550C660E770088129914AA16BB18CC12E
:10597000ADD1CEE1EFF13112100273325222B552A5
:105980009442F772D662399318837BB35AA3BDD37E
:105990009CC3FFF3DEE36224433420040114E66475
:1059A000C774A44485546AA54BB528850995EEE5CE
:1059B000CFF5ACC58DD55336722611163006D77685
:1059C000F6669556B4465BB77AA719973887DFF71E
:1059D000FEE79DD7BCC7C448E5588668A77840084D
:1059E000611802282338CCC9EDD98EE9AFF948896E
:1059F00069990AA92BB9F55AD44AB77A966A711AE5
:105A0000500A333A122AFDDBDCCBBFFB9EEB799BBD
:105A1000588B3BBB1AABA66C877CE44CC55C222C34
:105A2000033C600C411CAEED8FFDECCDCDDD2AAD0D
:105A30000BBD688D499D977EB66ED55EF44E133EC4
:105A4000322E511E700E9FFFBEEFDDDFFCCF1BBF5D
:105A50003AAF599F788F8891A981CAB1EBA10CD137
:105A60002DC14EF16FE18010A100C230E32004503F
:105A7000254046706760B9839893FBA3DAB33DC3B2
:105A80001CD37FE35EF3B1029012F322D23235428F
:105A9000145277625672EAB5CBA5A89589856EF542
:105AA0004FE52CD50DC5E234C324A01481046674DF
:105AB000476424540544DBA7FAB79987B8975FE792
:105AC0007EF71DC73CD7D326F2369106B01657662F
:105AD0007676154634564CD96DC90EF92FE9C8991A
:105AE000E9898AB9ABA94458654806782768C0187F
:105AF000E1088238A3287DCB5CDB3FEB1EFBF98BF2
:105B0000D89BBBAB9ABB754A545A376A167AF10ACE
:105B1000D01AB32A923A2EFD0FED6CDD4DCDAABD01
:105B20008BADE89DC98D267C076C645C454CA23C1E
:105B3000832CE01CC10C1FEF3EFF5DCF7CDF9BAFD1
:105B4000BABFD98FF89F176E367E554E745E932E6E
:105B5000B23ED10EF01E00002200250034004600A7
:105B60004B0059006C007A0088008E00920096006D
:105B70009A009E00A100A40020010D10030C110C3E
:105B80000C04020202020101010080F186F187F19A
:105B900088F18AF18CF190F191F198F199F110FE70
:105BA00011FE12FE13FE14FE15FE16FE000000008C
:105BB00000000100010101010101010101000000DB
:105BC0001300210027002B002F00330037003A007C
:105BD0003D0011000C00040002000200020002005F
:105BE00001000100010090F198F199F110FE11FE01
:105BF00012FE13FE14FE15FE16FE1011222E273E75
:105C00003128853436377F00285C000800000020EA
:105C1000600100004C0200087C5C0008600100206C
:105C200088280000825500081184A24A0400093324
:105C30000102030406070809293B693F0515020410
:105C40000608EA1F35017B138D3F1B08BD041AE1CE
:105C5000041391401B08010413AD411B08C5081A29
:105C60005D041AD10C1AF9081A39081A790413D5E7
:0C5C70004F0914D50A15801871000000BF
:04000005080001519D
